:020000040000FA
:1000000000008312073099000D309F00831658308E
:100010009F00FB30850081138312951615149514EB
:1000200000308500103062208D207620A200851AD5
:1000300022289F149F181A281E08A200A20EA20CA4
:1000400022087D200730220582072D2838284428E1
:10005000512832283E284A28512805080339013EF4
:1000600085002D2805080339013E043A8500322811
:1000700005080339031D04308500382805080339B5
:100080000319043085003E280508013E0339023E6D
:10009000850044280508013E0339023A023E8500E6
:1000A0004A28A401050803395D2022196720221D72
:1000B0006220A409240885005228820702340534EE
:1000C0000A341434A5006D20A50B63280800A6008F
:1000D00064306220A60B68280800C6300000FF3E8E
:1000E000031D6E28000000000000080003018316B5
:1000F0009B001C141A0883120800220883169B0117
:1001000083169A001C1555309D00AA309D009C1442
:1001100083128C1F89288C13080001307720813AC4
:10012000031D982802307720693A031D982800346F
:1001300083160030A2007D20831601309B008130A1
:10014000802083169B0A693080208312FF3450344C
:100150006534743465342034473472346934663419
:10016000663469347434683473342034323430344F
:100170003034363420342D34203452343134303459
:0E01800030343434303437342E3430343134AB
:02400E00843FED
:00000001FF
